:100000000C9463010C94CF160C94FC160C948B0189
:100010000C948B010C948B010C948B010C943B146D
:100020000C948B010C948B010C948B010C948B0120
:100030000C948B010C948B010C948B010C948B0110
:100040000C943B170C948B010C9495110C94DC11BF
:100050000C948B010C948B010C948B010C948B01F0
:100060000C948B010C948B010000004A616E466574
:10007000624D61724170724D61794A756E4A756C5C
:100080004175675365704F63744E6F7644656300C6
:1000900000004D6F6E5475655765645468754672FF
:1000A0006953617453756E00050A0D494C001F1C9D
:1000B0001F1E1F1E1F1F1E1F1E1F0101000100000B
:1000C0000C1E6307173BECFF8C0091038B03850329
:1000D0007E03780371036A0362035B0353034B03DC
:1000E00043033A0332032903200316030D030303DA
:1000F000F902EF02E402DA02CF02C402B902AE0250
:10010000A30297028C028002750269025D0251020D
:1001100046023A022E02220216020B02FF01F401ED
:10012000E801DD01D101C601BB01B001A6019B01BF
:10013000900186017C01720168015E0155014C014C
:1001400043013A0131012801200118011001080181
:100150000101F900F200EB00E400DD00D700D1005E
:10016000CB00C500BF00B900B400AE00A900A400D8
:100170009F009B00960092008D0089008500810001
:100180007D007A00760073006F006C0069006600E5
:10019000630060005D005A00580055005300510094
:1001A0004E004C004A004800460044004200400017
:1001B0003E003C003B00390038003600350033007B
:1001C000320030002F002E002D002B002A002900C5
:1001D00028002700260025002400230022002100FB
:1001E000210020000701070704070007000007009F
:1001F00001010707050505050704040707000703B4
:1002000002070705050404070705050704070101A0
:10021000070000070705070704070701070505078B
:100220000040105000000000000000001F1F0000F0
:10023000000000000000001F1F0000001F1F001F23
:100240001F0000000000000000001F1F1F1F000013
:1002500000001F1F0000001F1F001F1F1F1F001F87
:100260001F001F1F0200000000240027002A0000BA
:10027000000000250028002B0000000000230026BD
:10028000002900040404040404040402020202021B
:10029000020303030303030102040810204080014A
:1002A00002040810200102040810200000000700CA
:1002B000020100000304060000000000000000002E
:1002C000640C42135D0C11241FBECFEFD4E0DEBFDF
:1002D000CDBF11E0A0E0B1E0EAEDF4E302C005908B
:1002E0000D92A43AB107D9F712E0A4EAB1E001C037
:1002F0001D92A23CB107E1F712E0C4ECD2E004C0C9
:100300002297FE010E94251AC03CD107C9F70E941E
:1003100029170C94601A0C940000CF93DF93BC0152
:100320008230910510F462E070E0A091C002B091BB
:10033000C102ED01E0E0F0E040E050E021C0888142
:1003400099818617970769F48A819B81309719F004
:100350009383828304C09093C1028093C002FE0104
:1003600034C06817790738F44115510519F084171E
:10037000950708F4AC01FE018A819B819C01E9018B
:100380002097E9F641155105A9F1CA01861B970B83
:10039000049708F4BA01E0E0F0E02AC08D919C9146
:1003A000119784179507F9F46417750781F412966D
:1003B0008D919C911397309719F09383828304C099
:1003C0009093C1028093C002FD0132964CC0CA01D5
:1003D000861B970BFD01E80FF91F6193719302973C
:1003E0008D939C9340C0FD01828193819C01D90132
:1003F0001097A1F68091BE029091BF02892B41F423
:1004000080916301909164019093BF028093BE023A
:1004100040916501509166014115510541F44DB778
:100420005EB78091610190916201481B590B209148
:10043000BE023091BF02CA01821B930B8617970739
:1004400080F0AB014E5F5F4F8417950750F0420F6D
:10045000531F5093BF024093BE02F9016193719301
:1004600002C0E0E0F0E0CF01DF91CF910895CF939B
:10047000DF93009709F450C0EC0122971B821A8287
:10048000A091C002B091C102109709F140E050E084
:10049000AC17BD0708F1BB83AA83FE0121913191FE
:1004A000E20FF31FAE17BF0779F48D919C9111975E
:1004B000280F391F2E5F3F4F3983288312968D9165
:1004C0009C9113979B838A834115510571F4D093B6
:1004D000C102C093C00220C012968D919C911397C7
:1004E000AD01009711F0DC01D3CFFA01D383C283B1
:1004F00021913191E20FF31FCE17DF0769F4888154
:100500009981280F391F2E5F3F4FFA0131832083D5
:100510008A819B8193838283DF91CF910895FC012F
:1005200088279927E89421912032E9F3293010F0A7
:100530002E30C8F32B3241F02D3239F4689404C0C8
:100540000E94BD02820F911D219120532A30C0F3D9
:100550001EF4909581959F4F0895FB01DC0102C028
:1005600005900D9241505040D8F70895DC0101C02C
:100570006D9341505040E0F708957AE0979F902D99
:10058000879F802D910D11240895AEE0B0E0EBEC33
:10059000F2E00C94371A0D891E898F89988D97FF88
:1005A00002C080E090E801979E838D831A830983BF
:1005B00086E08C839E01255E3F4FCE010196698DBA
:1005C0007A8DA9010E9420034D815E8157FD0AC0EA
:1005D0002F813885421753070CF49A01020F131F1D
:1005E000F80110822E96E4E00C94531AAEE0B0E0CD
:1005F000ECEFF2E00C94371A8C0177FF02C060E058
:1006000070E8615070407E836D831A83098386E0B1
:100610008C83CE010196BA01A9010E9420032D818D
:100620003E8137FD09C0EF81F8852E173F070CF496
:10063000F901E00FF11F10822E96E4E00C94531A9A
:10064000ABE0B0E0E6E2F3E00C94291A3C012B01A8
:100650005A01FC0117821682838181FD03C06FEF6E
:100660007FEFC6C19AE0892E1E010894211C311C1F
:10067000F3012381F20123FD859123FF81912F0155
:10068000882309F4B2C1853239F423FD859123FF13
:1006900081912F01853229F490E0B3010E94130566
:1006A000E7CF982FFF24EE249924FFE1FF15D0F027
:1006B0009B3269F09C3228F4903259F0933291F4D5
:1006C0000EC09D3249F0903369F441E024C052E0FD
:1006D000F52A84E0F82A28C098E0F92A25C0E0E14C
:1006E000FE2A22C0F7FC29C0892F80538A3070F47B
:1006F000F6FE05C0989C902C1124980E15C0E89C1D
:10070000E02C1124E80EF0E2FF2A0EC09E3229F4FC
:10071000F6FC6BC140E4F42A07C09C3619F450E89B
:10072000F52A02C0983649F4F20123FD959123FF82
:1007300091912F01992309F0B8CF892F85548330E7
:1007400018F08052833038F444E050E0A40EB51E17
:100750005FE359830FC0933631F0933779F09335C7
:1007600009F056C020C0F5018081898342E050E045
:10077000A40EB51E610101E010E012C0F501C080B9
:10078000D180F6FC03C06FEF7FEF02C0692D70E0EF
:1007900042E050E0A40EB51EC6010E9408058C017F
:1007A0005FE7F52214C0F501C080D180F6FC03C0DC
:1007B0006FEF7FEF02C0692D70E042E050E0A40EC1
:1007C000B51EC6010E94FD048C0150E8F52AF3FE17
:1007D00007C01AC080E290E0B3010E941305EA94BA
:1007E0008E2D90E008171907A8F30EC0F601F7FC4C
:1007F0008591F7FE81916F0190E0B3010E9413058E
:10080000E110EA94015010400115110579F7EAC092
:10081000943611F0993669F5F7FE08C0F50120818C
:1008200031814281538184E090E00AC0F5018081EA
:1008300091819C01442737FD4095542F82E090E040
:10084000A80EB91E9FE6F92257FF09C050954095A2
:10085000309521953F4F4F4F5F4FE0E8FE2ACA0188
:10086000B901A1012AE030E00E943F05D82ED2183C
:1008700040C0953729F41F2D1F7E2AE030E01DC0AF
:100880001F2D197F9F3661F0903720F4983509F0BD
:10089000ACC00FC0903739F0983709F0A6C004C03B
:1008A00028E030E00AC0106114FD146020E130E05F
:1008B00004C014FD166020E132E017FF08C0F50106
:1008C000608171818281938144E050E008C0F5012C
:1008D00080819181BC0180E090E042E050E0A40E74
:1008E000B51EA1010E943F05D82ED2188FE7F82E21
:1008F000F122F6FE0BC05EEFF522D91438F4F4FEB7
:1009000007C0F2FC05C08FEEF82202C01D2D01C009
:10091000192DF4FE0DC0FE01ED0DF11D8081803317
:1009200019F499EEF92208C01F5FF2FE05C003C05A
:100930008F2D867809F01F5F0F2DF3FC14C0F0FE99
:100940000FC01E1510F09D2C0BC09D2C9E0C911AF3
:100950001E2D06C080E290E0B3010E9413051F5FC8
:100960001E15C0F304C01E1510F4E11A01C0EE24D8
:1009700004FF0FC080E390E0B3010E94130502FF63
:100980001DC001FD03C088E790E00EC088E590E03F
:100990000BC0802F867891F001FF02C08BE201C06E
:1009A00080E2F7FC8DE290E0B3010E94130506C0DF
:1009B00080E390E0B3010E9413059A94D914C0F328
:1009C000DA94F101ED0DF11D808190E0B3010E94F8
:1009D0001305DD20A9F706C080E290E0B3010E9474
:1009E0001305EA94EE20C1F743CEF30166817781C7
:1009F000CB012B96E2E10C94451AFC010590615065
:100A000070400110D8F7809590958E0F9F1F089524
:100A1000FC016150704001900110D8F780959095CD
:100A20008E0F9F1F08950F931F93CF93DF938C0119
:100A3000EB018B8181FF1BC082FF0DC02E813F81A6
:100A40008C819D812817390764F4E881F98101932D
:100A5000F983E88306C0E885F985802F0995892BFD
:100A600031F48E819F8101969F838E8302C00FEFA8
:100A70001FEFC801DF91CF911F910F910895FA01E7
:100A8000AA27283051F1203181F1E8946F936E7FCD
:100A90006E5F7F4F8F4F9F4FAF4FB1E03ED0B4E0BE
:100AA0003CD0670F781F891F9A1FA11D680F791FFF
:100AB0008A1F911DA11D6A0F711D811D911DA11D10
:100AC00020D009F468943F912AE0269F1124301920
:100AD000305D3193DEF6CF010895462F4770405DBB
:100AE0004193B3E00FD0C9F7F6CF462F4F70405D6A
:100AF0004A3318F0495D31FD4052419302D0A9F7C5
:100B0000EACFB4E0A6959795879577956795BA95BE
:100B1000C9F700976105710508959B01AC010A2E84
:100B200006945795479537952795BA95C9F7620F5B
:100B3000731F841F951FA01D0895CF93DF93EC01B1
:100B400088810E944718BC01AB81BC812CEC30E04D
:100B500041E050E00EC0F9013297859194918617DB
:100B6000970794F0F901859194918617970764F49B
:100B700003C04A175B077CF329813A81240F351F94
:100B8000C901DF91CF9108954F5F5F4F2E5F3F4FB7
:100B9000F0CF0F931F938C01862FF801608360E0E4
:100BA0000E94C918E6ECF0E085919491F8019283D7
:100BB0008183E8ECF0E085919491F801948383833C
:100BC0001F910F910895FC0182E791E0918380834A
:100BD00062836E5F63831482158216821782108689
:100BE0000895FC018481882361F485818F3F49F455
:100BF000968187818095981721F486818093AA0138
:100C0000089580E00895FC0182810895FC0114821A
:100C10001582168217820895FC0182E791E0918384
:100C200080830895FC0182E791E091838083CF0166
:100C30000E9438170895CF92DF92EF92FF920F93A0
:100C40001F93CF93DF93EC018B810E945C196C01A1
:100C50000E9483177B018C018091A6019091A701CE
:100C6000A091A801B091A901A8019701281B390BF7
:100C70004A0B5B0BDA01C90126E0B695A79597955B
:100C800087952A95D1F7582F80916701813009F017
:100C900044C08091A40186508630B0F53091A50102
:100CA000832F869586958695843008F083E0432FC0
:100CB0004770503190F4FE01E80FF11D248181E06E
:100CC00090E0A0E0B0E004C0880F991FAA1FBB1FEE
:100CD0004A95D2F78095282312C0503288F4FE013D
:100CE000E80FF11D248181E090E0A0E0B0E004C0B5
:100CF000880F991FAA1FBB1F4A95D2F7282B248360
:100D00003F5F3093A50109C01092A50190E0852FA7
:100D10008052833008F491E0988710926701CD28C3
:100D200019F081E080936701E092A601F092A7019B
:100D30000093A8011093A9015093A401DF91CF91D2
:100D40001F910F91FF90EF90DF90CF900895FC01DD
:100D500087818F770895FC0180850895FC01818546
:100D60000895FC0182850895FC0183850895FC01A6
:100D700084850895FC0185850895CF93DF93542FD2
:100D8000EC01A0E0B0E01EC04F81FB01EA0FFB1FA9
:100D9000842F90E024E0959587952A95E1F79C01B2
:100DA000220F331F220F331F220F331F880F991F6B
:100DB000280F391F4F70420F408311962196A7309C
:100DC000B10511F0A51700F3DF91CF910895FC0153
:100DD0008AE791E0918380830895282F30E0E4E052
:100DE00035952795EA95E1F7A90173E0440F551F62
:100DF0007A95E1F7220F331F420F531F8F70840F34
:100E00000895282F6AE00E94CE19382F3295307F3E
:100E1000822F0E94CE19832F890F0895FC018AE743
:100E200091E091838083CF010E9438170895AF929B
:100E3000BF92CF92DF92EF92FF920F931F93DF93B7
:100E4000CF930F92CDB7DEB77C016983FC0183811C
:100E500061E00E94C91800E010E05E010894A11C46
:100E6000B11CF1E0CF2ED12CF5016081C601002E1E
:100E700002C0880F991F0A94E2F76823F701838163
:100E80000E940819F701828160E00E940819F701A9
:100E9000828161E00E9408190F5F1F4F0830110521
:100EA00019F70F90CF91DF911F910F91FF90EF9065
:100EB000DF90CF90BF90AF900895EF92FF920F9385
:100EC0001F938C01F62EE42EFC01828160E00E94CB
:100ED0000819F801848161E00E940819FEEFFF22E1
:100EE000C8016F2D0E941707C8016E2D0E941707B9
:100EF000F801848160E00E940819F801828160E0B5
:100F00000E9408191F910F91FF90EF900895FC0126
:100F1000842F662311F440E001C040EA90E0837022
:100F20009070880F991F880F991F2370282B422BD0
:100F3000CF0160E90E945D07089541E046276EE811
:100F40000E945D070895EF920F93CF93DF93EC011A
:100F5000862F6AE771E0798368838A834B832C83C9
:100F60000D83EE8261E00E94C9188C8161E00E94CD
:100F7000C9188A8160E00E9408198C8160E00E9493
:100F800008198E818F3F39F061E00E94C9188E8167
:100F900060E00E9408198D818F3F39F061E00E9466
:100FA000C9188D8161E00E940819DF91CF910F91DE
:100FB000EF900895AF92BF92CF92DF92FF920F937E
:100FC0001F93CF93DF938C01FC01838160E00E942B
:100FD000C918FF24C0E0D0E0B1E0AB2EB12CC12C89
:100FE000D12CF801828161E00E940819F801828108
:100FF00060E00E940819F80183810E945C19892B26
:1010000061F0D601C5010C2E04C0880F991FAA1FDC
:10101000BB1F0A94D2F7F82A0CC0D601C5010C2ECA
:1010200004C0880F991FAA1FBB1F0A94D2F780958E
:10103000F8222196C830D105A1F68F2DDF91CF91EE
:101040001F910F91FF90DF90CF90BF90AF900895C8
:10105000EF92FF920F931F93CF93DF938C01662340
:1010600019F497E0E92E02C083E0E82EF8018281AE
:1010700060E00E940819F801848161E00E9408196B
:10108000C8016FEB0E941707F02EE801C8010E940B
:10109000DA078F8321969E012F192E15B8F3F801D8
:1010A000848160E00E940819F801828160E00E945A
:1010B0000819DF91CF911F910F91FF90EF90089544
:1010C000EF92FF920F931F93CF93DF93EC01E62EE5
:1010D000F42E122F61E00E949D07812F8F710E94D4
:1010E0000107482FCE0166E80E945D078F2D6DE055
:1010F0000E94CE19892F0E940107482FCE0168E86F
:101100000E945D07402F477009F447E0CE016AE86E
:101110000E945D078E2D64E60E94CE19892F0E94E1
:101120000107482FCE016CE80E945D07CE0160E008
:101130000E949D07CE0160E00E942808DF91CF91B8
:101140001F910F91FF90EF900895DF92EF92FF9221
:101150000F931F938C01D62EE42EF22E61E00E9495
:101160009D078F2D6CE30E94CE19892F0E940107E5
:10117000482FC80160E80E945D078E2D6CE30E9435
:10118000CE19892F0E940107482FC80162E80E94EA
:101190005D078D2D68E10E94CE19892F0E940107FD
:1011A000482FC80164E80E945D07C80160E00E9402
:1011B0009D07C80160E00E9428081F910F91FF90D1
:1011C000EF90DF900895FF920F931F938C01F62EFE
:1011D000FC01828160E00E940819F801848161E0CD
:1011E0000E940819F1E0FF2AC8016F2D0E9417071D
:1011F000C8010E94DA07F82EF801848160E00E949D
:101200000819F801828160E00E9408198F2D1F9152
:101210000F91FF9008951F93CF93DF93EC01162F4A
:1012200061E80E94E308112319F0482F406802C0CA
:10123000482F4F77CE0160E80E945D07DF91CF9184
:101240001F910895DC0186E0489F402D112450E055
:1012500020E0922F960FFA01EC51FE4F34911C962C
:101260008C911C97981738F41296ED91FC91139776
:10127000E90FF11D30831B969C911B97960F920FDF
:10128000FA01E951FE4F34911C968C911C979817E6
:1012900038F41296ED91FC911397E90FF11D30830C
:1012A0002F5F4F5F5F4F2330A1F60895FC018485C7
:1012B000681730F40280F381E02DE60FF11D4083C2
:1012C00008950F931F938C0182E891E0F8019183B8
:1012D0008083828193810E943702F80113821282F7
:1012E0001F910F9108950F931F938C0182E891E055
:1012F000F80191838083828193810E943702F801F3
:1013000013821282C8010E9438171F910F9108950D
:10131000FC0144858281938170E050E00E94B60216
:101320000895DF93CF93CDB7DEB7ED81FE81DE0167
:10133000199664858281938170E04F8158859D0163
:101340000E94F602CF91DF910895DF93CF93CDB73E
:10135000DEB7AD81BE812F811C966C911C9726173C
:1013600088F4FE013A9630E012968D919C91139785
:1013700070E0621B730B820F931F488559859F0194
:101380000E94F602CF91DF9108950F931F938C0175
:10139000FC01858160E00E940819F801858161E007
:1013A0000E940819F801858160E00E94081984E60E
:1013B00090E00E9402181F910F9108958F929F92C2
:1013C000AF92BF92CF92DF92EF92FF920F931F9353
:1013D000DF93CF930F92CDB7DEB7982E892E698316
:1013E000442341F0862F90E024E0959587952A9537
:1013F000E1F78983892D982D9C01790100E010E0A7
:101400005E010894A11CB11C81E0C82ED12CF5010D
:101410006081C601002E02C0880F991F0A94E2F76E
:101420006823F70186810E9408190F5F1F4F0894F7
:10143000E11CF11C0430110551F7892D982D0E94F3
:10144000C5090F90CF91DF911F910F91FF90EF9001
:10145000DF90CF90BF90AF909F908F900895FF92B4
:101460000F931F938C01F62E41E00E94DE09C80104
:101470006F2D40E00E94DE091F910F91FF900895AB
:10148000FF920F931F938C01F62EFC01848161E083
:101490000E940819C8016F2D0E942F0A1F910F91F9
:1014A000FF900895FF920F931F938C01F62EFC017D
:1014B000848160E00E940819C8016F2D0E942F0AE4
:1014C0001F910F91FF90089560680E94520A08953D
:1014D000DF92EF92FF920F931F93CF93DF937C01E4
:1014E000142F052FD22E0E94640A212F302FC901FC
:1014F000EC0110E005C0C70169910E94400A1F5F1E
:101500001D15C8F3DF91CF911F910F91FF90EF90C0
:10151000DF9008951F93CF93DF93EC0110E012C08A
:10152000E12FF0E0E05EFD4FE4912B85129FC001BA
:1015300011244A815B81480F591FCE016E2F0E94F2
:10154000680A1F5F8A85181758F3DF91CF911F91A2
:101550000895662311F060E301C060E24111686004
:10156000211164600E94520A0895662311F06CE014
:1015700001C068E041116260211161600E94520A5D
:101580000895662311F066E001C064E041116160D6
:101590000E94520A0895DF92EF92FF920F931F93D9
:1015A000CF93DF937C01162F072FD42E61E040E00C
:1015B0000E94C10AC70160E40E94520A212F302F05
:1015C000C901EC0110E005C0C70169910E94400A01
:1015D0001F5F1D15C8F3DF91CF911F910F91FF90F1
:1015E000EF90DF90089562E00E94520A80ED97E04C
:1015F0000E940218089561E00E94520A80ED97E06F
:101600000E94021808950F931F938C0180E593ECBC
:101610000E940218F801848160E00E940819F80114
:10162000858160E00E940819C80160E341E00E94E2
:10163000DE0984E991E10E940218C80160E341E0FB
:101640000E94DE0984E991E10E940218C80160E36A
:1016500041E00E94DE0986E990E00E940218C8017C
:1016600060E241E00E94DE09C80160E041E020E064
:101670000E94A90AC80160E040E020E00E94B50A8B
:10168000C8010E94FB0AC80161E040E00E94C10A53
:10169000C8010E94F30A1F910F910895EF92FF92E3
:1016A0000F931F938C010E94030B80E490E00E9433
:1016B0008D01F82EE92E64E272E040E450E00E94D1
:1016C000AD02C8016F2D7E2D40E40E94CB0A8F2D04
:1016D0009E2D0E943702C80161E040E020E00E9498
:1016E000B50A1F910F91FF90EF9008956F927F922E
:1016F0008F92AF92CF92EF920F93DF93CF93CDB7AC
:10170000DEB73C01862F62E871E0F30171836083EC
:101710008483458326830783E086C18661E00E9437
:10172000C918F301858161E00E94C918F30186811F
:1017300061E00E94C918F301878161E00E94C91825
:10174000F301808561E00E94C918F301818561E0A1
:101750000E94C918F301A38682868A9C802C1124DA
:1017600083948486882D90E00E948D01F30182830A
:101770009383C30160E00E948809CF91DF910F91AC
:10178000EF90CF90AF908F907F906F900895FC0175
:101790008AE891E0918380830895FC018AE891E0D2
:1017A00091838083CF010E9438170895FC018281C4
:1017B00061E00E9408190895FC0182810E9497143B
:1017C0000895FC01828170E00E9469180895FC016F
:1017D000862F2AE831E031832083628361E00E9412
:1017E000C9180895FC0180810E9447180895FC01E2
:1017F000862F608360E00E94C91808958F92AF928F
:10180000CF92EF920F9381309105C1F56F5F7F4FBB
:1018100009F04DC08BEA91E06EE00E94F70B8CEA74
:1018200091E069E00E94E70B8FEA91E06AE00E9494
:10183000E70B82EB91E061E142E123E10FEFEE245F
:10184000EA940E94A30780EC91E06FE00E94C90532
:1018500085EC91E068E047E026E005E0E4E0EE2E6C
:1018600073E0C72E50E1A52E32E0832E0E94760B46
:1018700082ED91E060E00E94E30519C0892BB9F484
:101880006F5F7F4FA1F482ED91E00E940C0685EC22
:1018900091E00E94610982EB91E00E94E7068FEAE5
:1018A00091E00E94C70B8CEA91E00E94C70B0F9158
:1018B000EF90CF90AF908F90089580E090E06FEF21
:1018C0007FEF0E94FE0B089581E090E06FEF7FEFC5
:1018D0000E94FE0B08951F9311E01CC08DE792E05B
:1018E0000E94CE12982F8091F301882339F49093AF
:1018F000DD019B3579F41093F3010CC0E82FF0E083
:10190000E352FE4F90838F5F8093F301863111F491
:101910001092F3018DE792E00E949D12892BF1F65F
:101920001F910895CF92DF92EF92FF920F931F9332
:10193000CF93DF93882341F0F5ECEF2EF1E0FF2EFB
:10194000813009F0BFC058C085EC91E060E00E9492
:10195000880982EB91E00E94AE060E94ED06182FE6
:101960008D3008F01C50812F6AE00E94CE19492F5B
:1019700085EC91E063E00E9422091A3060F085EC6A
:1019800091E060E047E00E94560985EC91E060E15B
:1019900047E00E94560982EB91E00E94AB060E944C
:1019A000ED06182F6AE00E94CE19482F85EC91E0D1
:1019B00069E00E942209812F6AE00E94CE19492F16
:1019C00085EC91E06DE00E94220982EB91E00E949B
:1019D000A70680FF0CC085EC91E067E042E00E9422
:1019E000560985EC91E067E142E00E94560985ECDA
:1019F00091E00E948A0A46C1C70160E00E948809FE
:101A0000C7016EE044E00E945609C7016FE044E060
:101A10000E945609C7016EE147E00E945609C701BE
:101A20006FE144E00E94560980EC91E00E949D0520
:101A3000EC0164E670E00E94DA19CB016AE070E024
:101A40000E94DA19482FCE016AE070E00E94DA198C
:101A5000CB016AE070E00E94DA19182F442329F0C4
:101A6000C70162E00E94220902C0882329F0C70151
:101A700066E0412F0E942209CE016AE070E00E94D8
:101A8000DA19482F85EC91E06AE00E942209D7FF1D
:101A90000CC085EC91E060E044E00E94560985ECC2
:101AA00091E061E044E00E94560982EB91E00E94DF
:101AB000A70680FFE7C085EC91E06DE045EA0E9453
:101AC0005609E0C0C70160E00E94880982EB91E0FE
:101AD0000E94B7060E94ED06D82E82EB91E00E948C
:101AE000AE06082F82EB91E00E94AB06182F82EB26
:101AF00091E00E94A7062DB73EB72B5030400FB69D
:101B0000F8943EBF0FBE2DBFEDB7FEB73196ADB70F
:101B1000BEB71296FC92EE92119798E1928320E064
:101B200031E03483238305831682178310868187EF
:101B300012860E94A50913E0D19EB0011124CB01A9
:101B400081579F4FFC014491CB0180579F4FFC016F
:101B500034916F567F4FFB012491EDB7FEB731965C
:101B6000ADB7BEB71296FC92EE9211978DE08283CC
:101B70008FE091E0948383834583168237831086B8
:101B8000218712860E94A509EDB7FEB73B960FB6D6
:101B9000F894FEBF0FBEEDBF82EB91E00E94B40649
:101BA0000E94ED06819F90011124C90188599F4F21
:101BB000FC01C490C90187599F4FFC01D49026595C
:101BC0003F4FF901049182EB91E00E94B106182F7A
:101BD00082EB91E00E94BA062DB73EB72E503040FE
:101BE0000FB6F8943EBF0FBE2DBFEDB7FEB73196CE
:101BF000ADB7BEB71296FC92EE92119726E131E096
:101C000033832283C4821582D6821782008711868D
:101C100012871386848715860E949109EDB7FEB757
:101C20003E960FB6F894FEBF0FBEEDBF80EC91E07C
:101C30000E949D052DB73EB7295030400FB6F8944D
:101C40003EBF0FBE2DBFEDB7FEB73196ADB7BEB7E5
:101C50001296FC92EE92119720E1228329E231E064
:101C600034832383968385838FED90E090878783E9
:101C70000E94A509EDB7FEB739960FB6F894FEBFDE
:101C80000FBEEDBFDF91CF911F910F91FF90EF90AD
:101C9000DF90CF9008958BEA91E00E94F20B80389C
:101CA000910514F480E108958150924014F080EF82
:101CB000089580EB08950F931F938FEA91E00E949F
:101CC000D60B85EC91E00E944E0B8CEA91E060917E
:101CD0006B010E94E10B02EB11E0C80161E00E9480
:101CE0009D07C80160E042E023E00E948707C80129
:101CF00060E00E940B09C80160E00E949D07C801D6
:101D000060E00E94280882ED91E00E94030660E9ED
:101D100071E141E050E00E94AC168DE792E040ECAA
:101D200052E160E070E00E9417121F910F91089538
:101D30001F93182F6623D1F48091DB018823B1F023
:101D400017C08FEA91E06DE279E020E630E040E0F4
:101D500050E00E94DC0B60E870E080E090E00E94C0
:101D6000A9178FEA91E00E94D60B1150112349F771
:101D70001F9108956F927F928F929F92AF92BF9220
:101D8000CF92DF92EF92FF920F931F93DF93CF9347
:101D9000CDB7DEB7A8970FB6F894DEBF0FBECDBFA4
:101DA000A7EECA2EA1E0DA2EC6010E948F02682E8D
:101DB000C60103960E948F02782EC60106960E94E5
:101DC0008F02882E02EB11E0C801662D472D282DC9
:101DD0000E94A508C60109970E948F02982EC6018D
:101DE00006970E948F02A82EC60103970E948F02B9
:101DF000B82EC60109960E948F02E82EC801692DEF
:101E00004A2D2B2D0E2D0E94600886EF9FEFC80EE5
:101E1000D91E86E1D6011D928A95E9F782E061E03C
:101E20000E94980E83E0E89E700111246FE870E034
:101E3000CB018E0D9F1DFC0144910894E11CF11C07
:101E4000CB018E0D9F1DFC0134910894E11CF11C07
:101E50006E0D7F1DFB0124918DB79EB748970FB67D
:101E6000F8949EBF0FBE8DBFEDB7FEB731968E01C1
:101E70000F5F1F4FADB7BEB712961C930E9311970D
:101E800088E290E0938382838FE291E0958384835C
:101E900096821782A0861186B2861386648615867E
:101EA00076861786808A118A428B138A348B158A2C
:101EB000268B178A0E94C502EDB7FEB778960FB63B
:101EC000F894FEBF0FBEEDBF8DE792E0B8010E940F
:101ED000F013A8960FB6F894DEBF0FBECDBFCF911A
:101EE000DF911F910F91FF90EF90DF90CF90BF9007
:101EF000AF909F908F907F906F9008958F929F9258
:101F0000AF92BF92CF92DF92EF92FF920F931F9307
:101F1000DF93CF93CDB7DEB72D970FB6F894DEBF22
:101F20000FBECDBFDE011196EEE8F1E086E0019034
:101F30000D928150E1F782EB91E060E00E94280869
:101F4000B7E0EB2EF12CEC0EFD1E82EB91E0B70119
:101F500047E00E94BD0682EB91E06D854B852A85A6
:101F60000C850E94600882EB91E06985488520E03D
:101F70000E94A50885EC91E061E040E021E00E942C
:101F8000B50A81E060E00E94980E82EB91E061E08A
:101F90000E940B0910E0CC24C39457014E01089411
:101FA000811C911C82ED91E00E94F105082F88238D
:101FB000C9F382EB91E0B50147E00E94BD06003411
:101FC00051F0033461F0073071F4CC2011F4DD24BA
:101FD0000CC0CC2408C0115030F416E004C01F5FC0
:101FE000163009F410E0DD24D394E12EFF24F7012C
:101FF000E654FF4F5491F701E054FF4F44913B8565
:10200000E32FF0E0E355FF4F24918D8590E083703E
:102010009070892B19F4323009F42F5F113011F4CC
:10202000922F01C0942FF401E10FF11D8081A82FA0
:10203000B0E0F501EA0FFB1FE081093019F005312E
:1020400061F405C0EF5F9E1740F4E52F06C0E15034
:10205000E51710F0EF3F09F4E92FAA0DBB1DEC9333
:102060003B85E32FF0E0E355FF4F24918D8590E011
:1020700083709070892B19F4323009F42F5F8A85B0
:10208000281708F42A8782EB91E06D854B852A8515
:102090000C850E94600882EB91E06985488520E00C
:1020A0000E94A50882EB91E060E00E94280882E08F
:1020B0000E94920C85EC91E00E948A0A87EA90E0E7
:1020C000E80EF91EF701649185EC91E00E94640A24
:1020D00082ED91E00E94060681E060E00E94980E89
:1020E000DD2009F05FCF82EB91E060E00E940B09F8
:1020F00085EC91E061E040E020E00E94B50A10929A
:102100006A0182E08093DC012D960FB6F894DEBF61
:102110000FBECDBFCF91DF911F910F91FF90EF9038
:10212000DF90CF90BF90AF909F908F90089582EDF9
:1021300091E00E94F105882309F496C0893109F4E1
:1021400046C08A3180F4893009F452C08A3020F4C4
:10215000873009F081C073C08D3009F442C08531E9
:1021600009F07AC055C0853469F0863420F484348F
:1021700009F072C060C0863409F452C0873409F097
:102180006BC060C01092690180916801882359F08A
:1021900085EC91E060E040E020E00E94B50A8CEA26
:1021A00091E06FEF0BC085EC91E061E040E020E052
:1021B0000E94B50A8CEA91E060916B010E94E10BEC
:1021C0008091680191E089278093680145C0109251
:1021D00069010E944B0E682F80936B018CEA91E09D
:1021E00014C08091690191E089278093690134C00E
:1021F0001092690180916B01813118F080528093B7
:102200006B018CEA91E060916B010E94E10B24C0AC
:102210001092690180916B01803F98F7805EEFCF4B
:1022200010926A018091DC018F5F63E00E94CE19F9
:102230009093DC0111C081E080936A010DC00E947F
:102240007E0F0AC08091DB0191E089278093DB013A
:1022500081E061E00E94980E82ED91E00E94060606
:1022600081E060E00E94980E08951F9382EB91E058
:1022700060E00E9428081091F40182EB91E00E9436
:10228000A7061817E9F180916A01882371F082EBA3
:1022900091E00E94A7060E94ED066AE00E94CE1916
:1022A00063E00E94CE199093DC018091DC010E94D2
:1022B000920C85EC91E00E948A0A80916901882342
:1022C00049F00E944B0E682F80936B018CEA91E0DD
:1022D0000E94E10B82EB91E00E94A706893551F440
:1022E00082EB91E00E94AB06893521F482E060E048
:1022F0000E94980E82EB91E00E94A7068093F40161
:1023000060EF70E080E090E00E94A9170E949710B3
:102310008091F2018D3511F40E94BA0E1F9108953B
:1023200082ED91E00E941B0608951F920F920FB656
:102330000F9211242F933F934F938F939F93EF937B
:10234000FF934091C60020913502309136022F5FF5
:102350003F4F2F73307080913702909138022817C9
:10236000390759F0E0913502F0913602EB50FE4FFB
:1023700040833093360220933502FF91EF919F9175
:102380008F914F913F912F910F900FBE0F901F9003
:102390001895E0918902F0918A02E05CFF4F8191EB
:1023A000919120813181821B930B8F739070892BC7
:1023B00011F00E946B0C08951F920F920FB60F92AE
:1023C00011242F933F938F939F93EF93FF9320912B
:1023D000790230917A0280917B0290917C022817D9
:1023E000390731F48091C1008F7D8093C10014C002
:1023F000E0917B02F0917C02E75CFD4F20818091AF
:102400007B0290917C0201968F73907090937C0276
:1024100080937B022093C600FF91EF919F918F9153
:102420003F912F910F900FBE0F901F901895AF9274
:10243000BF92DF92EF92FF920F931F93CF93DF93A0
:10244000EC017A018B01DD24403081EE580780E0F9
:10245000680780E0780711F0DD24D39491E0A92E7D
:10246000B12CEC89FD89DD2069F0C5010E8C02C01C
:10247000880F991F0A94E2F7808360E079E08DE38A
:1024800090E005C0108260E874E88EE190E0A80159
:1024900097010E94ED192150304040405040569520
:1024A00047953795279580E12030380720F0DD20CB
:1024B00011F0DD24D6CFE889F9893083EA89FB89D8
:1024C0002083EE89FF89408121E030E0C9010A8C38
:1024D00002C0880F991F0A94E2F7482B4083EE89C7
:1024E000FF894081C9010B8C02C0880F991F0A9493
:1024F000E2F7482B4083EE89FF894081C9010C8CAB
:1025000002C0880F991F0A94E2F7482B4083EE8996
:10251000FF8980810D8C02C0220F331F0A94E2F7DD
:10252000209528232083DF91CF911F910F91FF9059
:10253000EF90DF90BF90AF900895DC011C96ED9175
:10254000FC911D97E05CFF4F219131918081918139
:10255000281B390B2F733070C9010895DC011C96BC
:10256000ED91FC911D97E05CFF4F20813181E0549B
:10257000F040DF01AE5BBF4F8D919C911197281702
:10258000390719F42FEF3FEF07C08D919C91E80FA9
:10259000F91F8081282F30E0C9010895DC011C96C5
:1025A000ED91FC911D97E05CFF4F20813181E0545B
:1025B000F040DF01AE5BBF4F8D919C9111972817C2
:1025C000390719F42FEF3FEF10C08D919C911197AF
:1025D000E80FF91F20818D919C91119701968F73BF
:1025E000907011969C938E9330E0C9010895FC0180
:1025F00086859785DC01A05CBF4FFC01EE5BFF4F39
:102600002D913C9111978081918128173907C1F74D
:102610000895CF93DF93EC01EE85FF85E05CFF4FDB
:1026200020813181E054F0402F5F3F4F2F73307095
:10263000DF01AE5BBF4F8D919C9111972817390731
:10264000D1F3E05CFF4F80819181E054F040E80FCE
:10265000F91F6083EE85FF85E05CFF4F31832083A7
:10266000EE89FF89208181E090E00D8C02C0880F07
:10267000991F0A94E2F7282B208381E090E0DF91F4
:10268000CF9108951092800210927F0288EE93E01D
:10269000A0E0B0E08093810290938202A093830235
:1026A000B093840288E991E090937E0280937D024A
:1026B00085EF91E090938A028093890289E392E00A
:1026C00090938C0280938B0285EC90E090938E0225
:1026D00080938D0284EC90E09093900280938F021F
:1026E00080EC90E0909392028093910281EC90E0D4
:1026F000909394028093930286EC90E090939602DC
:102700008093950284E08093970283E080939802FF
:1027100087E08093990285E080939A0281E080931C
:102720009B020895CF92DF92EF92FF920F931F9337
:10273000CF93DF937C016B018A01C0E0D0E00FC032
:10274000D6016D916D01D701ED91FC910190F08161
:10275000E02DC7010995C80FD91F01501040011580
:10276000110571F7CE01DF91CF911F910F91FF906D
:10277000EF90DF90CF900895EF92FF920F931F9309
:102780008C01DC01ED91FC910190F081E02D6DE078
:1027900009957C01D801ED91FC910190F081E02D2B
:1027A000C8016AE009959C012E0D3F1DC9011F91CA
:1027B0000F91FF90EF900895CF93DF93DB010D9081
:1027C0000020E9F71197A61BB70BEC01E881F9810E
:1027D0000280F381E02DAD010995DF91CF9108953D
:1027E000EF92FF920F931F937C010E94DC138C01E8
:1027F000C7010E94BC13080F191FC8011F910F9138
:10280000FF90EF900895813041F0813018F08230D0
:10281000D1F409C010926E00089580916F008D7FF1
:1028200080936F000895809170008D7F8093700079
:1028300081E08093B0008091B100887F84608093B4
:10284000B1001092B30008951F93182F80916C016E
:10285000811711F09FEF06C0E4E6F2E094918FEF4C
:1028600080936C01892F0E940314812F60E00E94E5
:1028700008191F9108951F920F920FB60F921124FD
:102880002F933F934F935F936F937F938F939F9378
:10289000AF93BF93EF93FF938091AA029091AB0205
:1028A000A091AC02B091AD020097A105B10551F124
:1028B000E091AE02F091AF0280819091B002892741
:1028C00080838091AA029091AB02A091AC02B0915A
:1028D000AD02181619061A061B06C4F48091AA0246
:1028E0009091AB02A091AC02B091AD020197A10909
:1028F000B1098093AA029093AB02A093AC02B0936B
:10290000AD0204C080916C010E942414FF91EF91EC
:10291000BF91AF919F918F917F916F915F914F91F7
:102920003F912F910F900FBE0F901F9018952F92EF
:102930003F925F926F927F928F929F92AF92BF92DF
:10294000CF92DF92EF92FF920F931F93DF93CF937B
:1029500000D000D0CDB7DEB7A82F1B0129833A8362
:102960004B835C8380916C018A1721F4E4E6F2E0EA
:10297000549082C08F3F09F0D9C1A0936C01E4E666
:10298000F2E054902FEF521609F4D0C181E05816AE
:1029900039F192E0591609F449C0552009F06CC08C
:1029A00014BC15BC84B5826084BD85B5816085BDCD
:1029B0002A2F30E0F901ED57FD4FE491F0E0EE0FE2
:1029C000FF1FE159FD4F859194919093A10280934F
:1029D000A00229563D4FF90184918093A2024EC076
:1029E0001092800010928100809181008860809315
:1029F0008100809181008160809381002A2F30E0E6
:102A0000F901ED57FD4FE491F0E0EE0FFF1FE159A2
:102A1000FD4F859194919093A8028093A702295627
:102A20003D4FF90184918093A90228C01092B00013
:102A30001092B1008091B00082608093B0008091CC
:102A4000B10081608093B1002A2F30E0F901ED5789
:102A5000FD4FE491F0E0EE0FFF1FE159FD4F85912E
:102A600094919093AF028093AE0229563D4FF901A5
:102A700084918093B00202C057FC58C18A2F61E054
:102A80000E94C918552021F0F2E05F1609F0BDC080
:102A900031018824992460E072E18AE790E0A40182
:102AA00093010E94ED1959016A018601750108948C
:102AB000E108F108010911092FEFE216F1040105FF
:102AC000110509F008F498C060E472E48FE090E02A
:102AD000A40193010E94ED1979018A010894E1088B
:102AE000F1080109110982E05816C1F49FEFE916B7
:102AF000F1040105110509F008F483C060E970EDE7
:102B000083E090E0A40193010E94ED1979018A010C
:102B10000894E108F1080109110983E0AFEFEA1612
:102B2000F1040105110509F008F467C068E478EEC6
:102B300081E090E0A40193010E94ED1979018A01DE
:102B40000894E108F10801091109552011F483E006
:102B50001DC0B2E05B1611F084E018C0EFEFEE1676
:102B6000F1040105110509F008F4DEC064E274EF18
:102B700080E090E0A40193010E94ED1979018A019F
:102B80000894E108F1080109110985E0FFEFEF164B
:102B9000F1040105110589F180F162E17AE780E035
:102BA00090E0A40193010E94ED1979018A01089433
:102BB000E108F10801091109552011F086E001C072
:102BC00084E02FEFE216F10401051105B1F0A8F041
:102BD000860175019AE016950795F794E7949A9502
:102BE000D1F70894E108F10801091109552011F005
:102BF00087E008C085E003C081E0552019F485BD59
:102C00003AC082E08093B10036C05101CC24DD246B
:102C100060E072E18AE790E0A60195010E94ED195B
:102C200079018A010894E108F1080109110980E09D
:102C3000E81680E0F80681E0080780E0180710F445
:102C400091E010C068E478EE81E090E0A601950183
:102C50000E94ED1979018A010894E108F10801093F
:102C6000110993E0A1E05A1631F480918100887F28
:102C7000982B9093810089819A81AB81BC810097C8
:102C8000A105B10529F48FEF9FEFAFEFBFEF13C0A0
:102C9000220C331CB10180E090E029813A814B8104
:102CA0005C810E94AF1928EE33E040E050E00E94C2
:102CB000ED19C901DA01E1E05E16A1F0F2E05F165C
:102CC00019F1552099F5E7BC80939C0290939D02E1
:102CD000A0939E02B0939F0280916E0082608093C9
:102CE0006E0024C0F0928900E09288008093A302D5
:102CF0009093A402A093A502B093A60280916F00C6
:102D0000826080936F0012C0E092B3008093AA02A9
:102D10009093AB02A093AC02B093AD02809170008F
:102D200082608093700002C084E06CCF0F900F909F
:102D30000F900F90CF91DF911F910F91FF90EF9027
:102D4000DF90CF90BF90AF909F908F907F906F90CB
:102D50005F903F902F900895823000F5E82FF0E0CB
:102D6000EE0FFF1FEF54FD4F71836083882319F02E
:102D70008130A1F408C0809169008C7F842B8093FE
:102D80006900E89A089580916900440F551F440F27
:102D9000551F837F842B80936900E99A08951F92C1
:102DA0000F920FB60F9211242F933F934F935F937F
:102DB0006F937F938F939F93AF93BF93EF93FF9303
:102DC0008091B1029091B202892B29F0E091B10279
:102DD000F091B2020995FF91EF91BF91AF919F9150
:102DE0008F917F916F915F914F913F912F910F90B4
:102DF0000FBE0F901F9018951F920F920FB60F9253
:102E000011242F933F934F935F936F937F938F93EF
:102E10009F93AF93BF93EF93FF938091B3029091F1
:102E2000B402892B29F0E091B302F091B402099524
:102E3000FF91EF91BF91AF919F918F917F916F9192
:102E40005F914F913F912F910F900FBE0F901F9068
:102E50001895CF93DF930E940C180E945B0EC9EC6B
:102E6000D1E10E9435112097E1F30E94C911F9CFF9
:102E70000E94370208951F920F920FB60F921124ED
:102E80002F933F938F939F93AF93BF938091B902FA
:102E90009091BA02A091BB02B091BC023091BD02E8
:102EA0000196A11DB11D232F2D5F2D3720F02D5729
:102EB0000196A11DB11D2093BD028093B90290938C
:102EC000BA02A093BB02B093BC028091B50290916C
:102ED000B602A091B702B091B8020196A11DB11D32
:102EE0008093B5029093B602A093B702B093B80254
:102EF000BF91AF919F918F913F912F910F900FBEF6
:102F00000F901F9018959FB7F8942091B5023091BB
:102F1000B6024091B7025091B80286B5A89B06C090
:102F20008F3F21F02F5F3F4F4F4F5F4F9FBF542F79
:102F3000432F322F2227280F311D411D511D82E0C2
:102F4000220F331F441F551F8A95D1F7B901CA01BB
:102F500008959B01AC017FB7F8948091B5029091E0
:102F6000B602A091B702B091B80266B5A89B05C0A1
:102F70006F3F19F00196A11DB11D7FBFBA2FA92F78
:102F8000982F8827860F911DA11DB11D62E0880F23
:102F9000991FAA1FBB1F6A95D1F7BC012DC0FFB7AF
:102FA000F8948091B5029091B602A091B702B091C9
:102FB000B802E6B5A89B05C0EF3F19F00196A11D28
:102FC000B11DFFBFBA2FA92F982F88278E0F911DF3
:102FD000A11DB11DE2E0880F991FAA1FBB1FEA9532
:102FE000D1F7861B970B885E9340C8F22150304082
:102FF0004040504068517C4F211531054105510535
:1030000071F60895019739F0880F991F880F991F5D
:1030100002970197F1F70895789484B5826084BD92
:1030200084B5816084BD85B5826085BD85B58160CC
:1030300085BDEEE6F0E0808181608083E1E8F0E02C
:103040001082808182608083808181608083E0E85B
:10305000F0E0808181608083E1EBF0E0808184603A
:103060008083E0EBF0E0808181608083EAE7F0E03C
:1030700080818460808380818260808380818160A0
:1030800080838081806880831092C1000895982F8A
:103090008E3008F09E50977080916D018295880F58
:1030A000880F807C892B80937C0080917A008064DB
:1030B00080937A0080917A0086FDFCCF2091780081
:1030C00040917900942F80E030E0282B392BC90102
:1030D00008951F93CF93DF93182FEB0161E00E94B7
:1030E000C918209709F44AC0CF3FD10509F449C057
:1030F000E12FF0E0E555FD4F84918330C1F084303D
:1031000028F4813051F08230B1F50CC0863019F1CD
:10311000873049F1843079F514C084B5806884BD66
:10312000C7BD33C084B5806284BDC8BD2EC0809148
:103130008000806880938000D0938900C0938800CD
:1031400024C080918000806280938000D0938B00A7
:10315000C0938A001AC08091B00080688093B0004C
:10316000C093B30012C08091B00080628093B00021
:10317000C093B4000AC0C038D1051CF4812F60E0B0
:1031800002C0812F61E00E940819DF91CF911F9149
:103190000895CF93DF93482F50E0CA0189569D4F81
:1031A000FC0134914D575D4FFA018491882369F1F8
:1031B00090E0880F991FFC01EB59FD4FA591B49148
:1031C000FC01E159FD4FC591D491662351F42FB70D
:1031D000F8948C91932F909589238C9388818923DF
:1031E0000BC0623061F42FB7F8948C91932F9095B7
:1031F00089238C938881832B88832FBF06C09FB738
:10320000F8948C91832B8C939FBFDF91CF9108957D
:10321000482F50E0CA0185559D4FFC012491CA01F9
:1032200089569D4FFC0194914D575D4FFA013491A1
:10323000332309F440C0222351F1233071F02430AC
:1032400028F42130A1F0223011F514C02630B1F05D
:103250002730C1F02430D9F404C0809180008F77EA
:1032600003C0809180008F7D8093800010C084B562
:103270008F7702C084B58F7D84BD09C08091B00076
:103280008F7703C08091B0008F7D8093B000E32FD3
:10329000F0E0EE0FFF1FE159FD4FA591B4912FB75C
:1032A000F894662321F48C919095892302C08C9127
:1032B000892B8C932FBF0895682F70E0CB01855523
:1032C0009D4FFC012491CB0189569D4FFC014491F7
:1032D0006D577D4FFB019491992319F420E030E064
:1032E0003CC0222351F1233071F0243028F42130E6
:1032F000A1F0223011F514C02630B1F02730C1F012
:103300002430D9F404C0809180008F7703C080916D
:1033100080008F7D8093800010C084B58F7702C0BD
:1033200084B58F7D84BD09C08091B0008F7703C0C4
:103330008091B0008F7D8093B000892F90E0880F3E
:10334000991F87589D4FFC01A591B4918C9120E065
:1033500030E0842311F021E030E0C9010895629F3C
:10336000D001739FF001829FE00DF11D649FE00D7D
:10337000F11D929FF00D839FF00D749FF00D659FDE
:10338000F00D9927729FB00DE11DF91F639FB00DDD
:10339000E11DF91FBD01CF0111240895991B79E0AA
:1033A00004C0991F961708F0961B881F7A95C9F7D5
:1033B0008095089597FB092E07260AD077FD04D043
:1033C0002ED006D000201AF4709561957F4F089595
:1033D000F6F7909581959F4F0895A1E21A2EAA1BAA
:1033E000BB1BFD010DC0AA1FBB1FEE1FFF1FA217B5
:1033F000B307E407F50720F0A21BB30BE40BF50BB2
:10340000661F771F881F991F1A9469F7609570953A
:10341000809590959B01AC01BD01CF010895AA1B39
:10342000BB1B51E107C0AA1FBB1FA617B70710F0AF
:10343000A61BB70B881F991F5A95A9F780959095E1
:10344000BC01CD010895EE0FFF1F0590F491E02D12
:1034500009942F923F924F925F926F927F928F9238
:103460009F92AF92BF92CF92DF92EF92FF920F9313
:103470001F93CF93DF93CDB7DEB7CA1BDB0B0FB61D
:10348000F894DEBF0FBECDBF09942A8839884888DA
:103490005F846E847D848C849B84AA84B984C88470
:1034A000DF80EE80FD800C811B81AA81B981CE0F67
:1034B000D11D0FB6F894DEBF0FBECDBFED0108954C
:1034C00012E0C4ECD2E004C0FE010E94251A22964C
:0A34D000C63CD107C9F7F894FFCFFE
:1034DA00253032783A253032783A2530327800254C
:1034EA006325632563002563256325632E25303212
:1034FA00782C323025303278002564256343005316
:10350A006574204461746554696D6520746F202563
:10351A003032642D253032642D2530326420253234
:10352A00643A2532643A253264202563256325638B
:10353A00002000C202000001010101F0FF010000A9
:10354A0000000C06120600000000E7060E07000045
:10355A0000006109730900000000C70BCD0B0403CA
:10356A000605020100000000091392139D12CE12F3
:04357A00AE12F71284
:103E0000112484B714BE81FFF0D085E08093810037
:103E100082E08093C00088E18093C10086E08093B7
:103E2000C20080E18093C4008EE0C9D0259A86E06C
:103E300020E33CEF91E0309385002093840096BB13
:103E4000B09BFECF1D9AA8958150A9F7CC24DD2404
:103E500088248394B5E0AB2EA1E19A2EF3E0BF2E27
:103E6000A2D0813461F49FD0082FAFD0023811F076
:103E7000013811F484E001C083E08DD089C0823420
:103E800011F484E103C0853419F485E0A6D080C024
:103E9000853579F488D0E82EFF2485D0082F10E0EE
:103EA000102F00270E291F29000F111F8ED0680127
:103EB0006FC0863521F484E090D080E0DECF843678
:103EC00009F040C070D06FD0082F6DD080E0C816C8
:103ED00088E3D80618F4F601B7BEE895C0E0D1E053
:103EE00062D089930C17E1F7F0E0CF16F8E3DF0614
:103EF00018F0F601B7BEE89568D007B600FCFDCF14
:103F0000A601A0E0B1E02C9130E011968C911197C0
:103F100090E0982F8827822B932B1296FA010C01A0
:103F200087BEE89511244E5F5F4FF1E0A038BF07D0
:103F300051F7F601A7BEE89507B600FCFDCF97BE86
:103F4000E89526C08437B1F42ED02DD0F82E2BD092
:103F50003CD0F601EF2C8F010F5F1F4F84911BD0D7
:103F6000EA94F801C1F70894C11CD11CFA94CF0C53
:103F7000D11C0EC0853739F428D08EE10CD084E9ED
:103F80000AD08BE07ACF813511F488E018D01DD0AB
:103F900080E101D065CF982F8091C00085FFFCCFD4
:103FA0009093C60008958091C00087FFFCCF809158
:103FB000C00084FD01C0A8958091C6000895E0E688
:103FC000F0E098E1908380830895EDDF803219F06E
:103FD00088E0F5DFFFCF84E1DECF1F93182FE3DF0A
:103FE0001150E9F7F2DF1F91089580E0E8DFEE2736
:043FF000FF2709940A
:023FFE000404B9
:0400000300003E00BB
:00000001FF
